:020000040000FA
:100000000000831603130301880083120313880181
:100010008A28F930A0000000A00B0B280800A100DE
:100020000920A10B10280800081509200811092033
:100030000800A500F0398800A418881414200920AD
:10004000A50E2508F0398800A4188814142009206A
:100050000800820743344F344E34533454343A3416
:100060003034313432343334343435343634373454
:1000700038343934820756344134523449344134A7
:1000800042344C34453420343D34203464300F2025
:10009000F030A40030308800142005300F201420E8
:1000A00009201420081214202830192008301920A3
:1000B0000130192006301920803019200C30192009
:1000C0000800A301A414230829201920A30A230847
:1000D000103C031D6328C030A4101920A30123087D
:1000E0003A20A4141920A30A23080B3C031D6F28EF
:1000F0000800A2013030A2072208A4141920CB3036
:10010000A4101920FA300F20A20A22083A3C031D3D
:0A0110007C28792846206120792818
:02400E00313748
:00000001FF
